:1000000019C033C032C031C030C02FC02EC02DC087
:100010002CC02BC02BC029C028C027C026C025C09B
:1000200024C023C022C021C020C01FC04CC01DC09E
:100030001CC01BC011241FBECFEFCDBFDFE3DEBF4E
:100040001FE3A0E0BFE3E7EEF4E002C005900D92ED
:10005000A230B107D9F72FE3A2E0BFE301C01D92A0
:10006000A232B207E1F77FD138C2CACF1F920F92F6
:100070000FB60F9211248F938091123F811103C00C
:1000800082E0809306048091163F811103C080E4D2
:100090008093060480911A3F811103C088E0809309
:1000A000060480911E3F811103C084E08093060402
:1000B00080E180930B0A10920A0A8F910F900FBE75
:1000C0000F901F9018951F920F920FB60F92112448
:1000D0000F931F932F933F934F935F936F937F9350
:1000E0008F939F93AF93BF93CF93DF93EF93FF9340
:1000F00080910008982F987F983F09F0B3C08A3FFD
:1001000009F492C0B8F4883F21F1FF91EF91DF919B
:10011000CF91BF91AF919F918F917F916F915F919F
:100120004F913F912F911F910F910F900FBE0F9004
:100130001F9018958B3F09F491C08C3F31F7809147
:10014000033F811103C08EE4809306041092033FA5
:10015000DCCF8091033F8823C1F28091023F81115F
:1001600040C08091200A9091210A969587958093AE
:10017000003F9093013F8091003F9091013F809319
:10018000280A9093290A1092200A1092210A80E1ED
:1001900080930B0A80930A0A30E020E0E901CC0F3B
:1001A000DD1FCC0FDD1FFE01EE5EF04C8381882346
:1001B00019F0838181508383FE01EE5EF04C8381D0
:1001C000811109C08081811110C0F901ED51FB47F7
:1001D0008081809305042F5F3F4F24303105F1F675
:1001E00094CF81508093023FC6CF6081828190E09E
:1001F00070E06F5F7F4F4AD182838281882341F014
:1002000042818081869590E001964817190631F465
:10021000F901ED51FB47808180930704CE5ED04CFD
:100220008A818F5F8A83D7CF1092200A1092210A89
:1002300090E080E0FC01EE0FFF1FEE0FFF1FEE5E6F
:10024000F04C12822181238301968430910591F72D
:1002500082E08093023F8EE48093060481E08093E5
:10026000033F53CF87FF6FC0803F29F0873F49F09E
:100270001092113F4ACF8093053F81E08093113F58
:1002800044CF8091113F8B3099F7E5E0FFE3AEED6D
:10029000B4E88AE09FE331912D913213E9CF8E17B4
:1002A0009F07C9F780910A3F9091043F891711F089
:1002B0008F37F1F680910B3F8032D1F680910C3F61
:1002C0008111D6CFC0910E3FC43090F660910F3FA0
:1002D00080910D3F8A3221F150F4893249F684E051
:1002E000C89FE0011124CE5ED04C6883C1CF813419
:1002F000F9F08F3709F0BCCFD0E08E01000F111F4D
:10030000000F111F0E5E104CF8016081CC0FDD1F35
:10031000CE0101969CD0F8016181CE01029611C0F8
:10032000E4E0CE9FE0011124CE5ED04C6983A0CFE3
:100330008FEF860F8E3708F09BCF6093043F90E0DD
:1003400080E085D095CFE091113F9FEF9E0F9B30CD
:1003500008F0DBCE91E09E0F9093113FF0E0EB5F51
:10036000F04C8083D2CEF894C1E088ED84BFC09376
:10037000610090E080E063D08093043F8F3F31F4D0
:10038000C093043F61E090E080E061D001E010E0C4
:10039000F12CE12CC80153D0E701CC0FDD1FCC0FAD
:1003A000DD1FCE5ED04C888368018FEFC81AD80A53
:1003B000C60145D0898388818F3F41F41882198214
:1003C0006881C80144D06981C60141D08FEFE81A25
:1003D000F80A0E5F1F4F84E0E816F104D9F68FE7A4
:1003E000809300041092040410920102809117047B
:1003F000877F8093170480E094E0809308089093AF
:10040000090880E8809305088093060883E08093BC
:1004100007081092000A8FE08093050A8FEF9FEF84
:100420008093260A9093270A80E898E18093280A0F
:100430009093290A8DE08093000A7894FFCF03D02F
:10044000808199270895FC01E050FC4E0895262FE5
:100450000E9423020080021619F00E9433020197C5
:1004600001970895262FAF93BF93E0E0F0E132812A
:1004700031FDFDCFDC01A050BC4E2C932DE924BFF3
:1004800023E020830196BF91AF91089597FB072E3B
:1004900016F4009406D077FD08D00BD007FC05D0E9
:1004A0003EF4909581959F4F0895709561957F4F8B
:1004B0000895AA1BBB1B51E107C0AA1FBB1FA617AB
:1004C000B70710F0A61BB70B881F991F5A95A9F7FD
:0E04D00080959095BC01CD010895F894FFCF62
:0904DE00F00020131A024008048A
:0204E70080187B
:00000001FF
